:1018000012C02BC02AC029C028C027C026C025C0AE
:1018100024C023C022C021C020C01FC01EC01DC0C4
:101820001CC01BC01AC011241FBECFE5D4E0DEBF10
:10183000CDBF10E0A0E6B0E0EEE9FEE102C0059009
:101840000D92A036B107D9F711E0A0E6B0E001C0D3
:101850001D92A43AB107E1F7F1C2D2CF0F93EF93F3
:10186000FF933ED0FC01062F35D0FF91EF910F91F1
:1018700008950F930F921F92EF93FF9331D0FC01C5
:101880000B0101E027D0FF91EF911F900F900F9176
:1018900008950F930F92EF93FF9322D0FC0160FD08
:1018A00067BFC895802DE395C895902DFF91EF9166
:1018B0000F900F9108950F930F9212D0082E09E008
:1018C00009D00F900F9108950F930AD001E102D033
:1018D0000F910895E199FECF07BFE895FFFF000043
:1018E00007B700FDFDCF089583E089B9549A539A54
:1018F00008958CB19927089540E050E048175907A2
:1019000050F42AE633E000002150304037FFFBCF8F
:101910004F5F5F4FF3CF08958BB199278078907018
:101920000895549853980895FCDF0EC308958CB918
:101930005E9BFECF5E9A0895EFDF8823E9F3D9DF3F
:10194000803219F481E090E0089585E1F0DF80E0D5
:1019500090E008950895EF92FF920F931F93CF9315
:10196000DF937B01C0E0D0E0C617D70760F48C019D
:10197000D3DF8823E9F3BDDFF80181938F0121963E
:10198000CE15DF05A8F381E090E0DF91CF911F91A4
:101990000F91FF90EF90089590E0282F3327213882
:1019A000310589F02238310524F42038310549F019
:1019B0000DC02238310549F02839310539F493E05A
:1019C00005C092E003C091E001C092E1892F992700
:1019D000089540E050E06091A0007091A10046178A
:1019E0005707E8F4E2EAF0E08091A2018EBB809113
:1019F000A2019091A301292F33272FBB0196909329
:101A0000A3018093A20180818DBBE29AE19AE199C2
:101A1000FECF4F5F5F4F31964617570728F3089563
:101A20000F931F93CF93DF9300E010E08091A0000D
:101A30009091A10008171907D0F4C2EAD0E0809174
:101A4000A2019091A301880F991F60E0800F911F60
:101A500020DF8883892F992789830E5F1F4F229665
:101A60008091A0009091A1000817190740F3DF9121
:101A7000CF911F910F9108958091A0009091A100A6
:101A80000097C1F0E2EAF0E0AC018091A2018EBBC8
:101A90008091A2019091A301292F33272FBB01969A
:101AA0009093A3018093A201E09A8DB3819341505A
:101AB000504059F708950F931F93CF93DF938C01F4
:101AC0006115710539F0EB01F80181918F012FDF6C
:101AD0002197D1F781E090E0DF91CF911F910F9195
:101AE0000895EF92FF920F931F93CF93DF93C0E07F
:101AF000D0E08E017E01CFE7D0E0F092A301E0922A
:101B0000A20163E0C801AADE219780E290E0E80E1E
:101B1000F91E005C1F4FD7FFF0CFD6DEDF91CF91CB
:101B20001F910F91FF90EF900895EF92FF920F9306
:101B30001F93CF93DF9300E010E08091A00090917D
:101B4000A1000817190708F043C0EE24FF24E8019C
:101B5000CD55DF4FF801EE55FF4FEE0DFF1D4081D3
:101B6000888122969927382F2227240F311D8091B2
:101B7000A2019091A301880F991FB9018E0D9F1D9D
:101B800078DE82E090E0E80EF91E90E4E916F104B8
:101B900008F38091A2019091A301880F991F63E03F
:101BA000800F911F5BDE8091A2019091A301880FAD
:101BB000991F65E0800F911F51DE86DE005C1F4F8C
:101BC0008091A0009091A1000817190708F4BDCFDB
:101BD000DF91CF911F910F91FF90EF900895CF93D8
:101BE000C0E069E081E090E054DE84FF02C08F7EB7
:101BF00062DE92DE8823E9F37CDE99278235910547
:101C0000DCF4803591050CF04CC08134910509F469
:101C100050C0823491053CF48033910509F441C0F1
:101C2000C19759F108C18234910509F451C0853436
:101C3000910509F450C0FFC08635910509F4CAC06A
:101C4000873591054CF48235910509F451C08535ED
:101C5000910509F453C0EFC08437910509F487C09A
:101C6000853791052CF48436910509F45EC0E3C0F4
:101C70008537910509F4A2C0DEC05EDE882309F431
:101C8000B8CF84E154DE81E452DE86E550DE82E5A1
:101C90004EDE80E24CDE83E54ADE84E548DE8BE4FE
:101CA00005C04ADE882309F4A4CF84E140DE80E148
:101CB000C3C061E070E080E690E04DDE3DDE882349
:101CC00009F497CF84E133DE8091600065DEEECFCA
:101CD00064E170E009C061E070E080E690E03BDE26
:101CE000809160009927BC0180E690E034DED9CF76
:101CF00023DE882309F47DCFF4DED7CF62E070E0E5
:101D000080E690E028DE18DE882309F472CF209167
:101D10006000809161009927982F8827820F911D7C
:101D20009093A3018093A201C0CF63E070E080E6AE
:101D300090E011DE20916100809160009927982F3A
:101D40008827820F911D9093A1008093A000BC0171
:101D500082EA90E000DEF0DD882309F44ACF80912A
:101D60006200863411F4E1DEA0CF33DE9ECF63E063
:101D700070E080E690E0EFDD2091610080916000EE
:101D80009927982F8827820F911D9093A100809307
:101D9000A000D2DD882309F42CCF80916200863424
:101DA00011F43EDE01C068DE84E1C1DD6091A00077
:101DB0007091A10082EA90E07EDE79CFBDDD8823BC
:101DC00009F417CF84E1B3DD8EE1B1DD83E9AFDD46
:101DD00087E06CCF64E070E080E690E0BCDDACDDD5
:101DE000882309F406CF84E1A2DD8091600080356C
:101DF00031F480916100882361F4C82F17C08835C1
:101E000031F480916100883061F4C3E00FC0803507
:101E100031F480916100883049F4C2E007C0883510
:101E200029F480916100882309F4C1E069E08C2FD6
:101E300099272FDD3BCF85E17ADDDBCECFE5D4E0FE
:101E4000DEBFCDBFCEE1F8948EEF91E01FD0843B92
:101E500049F48FEF91E01AD0833C21F48DEF91E0AB
:101E600015D081BF41DD45DD84E690E045DD54DDE0
:101E7000882321F4C150C8BBCC23B1F7CC2311F087
:101E8000AEDE01C051DD80E090E008C0E199FECFF8
:0E1E90009FBB8EBBE09A99278DB30895FFCFBC
:0400000300001800E1
:00000001FF
